:020000040800F2
:100000008808002045010008510A0008490A000834
:100010004D0A00088D010008E71B000800000000E1
:100020000000000000000000000000008115000832
:100030002D09000800000000E10F0008E916000883
:100040005F0100085F0100085F0100085F01000810
:100050005F0100085F0100085F0100085F01000800
:100060005F0100085F0100085F0100085F010008F0
:100070005F0100085F0100085F0100085F010008E0
:100080005F0100085F0100085F0100085F010008D0
:100090005F0100085F0100085F0100085F010008C0
:1000A0005F0100085F0100085F0100085F010008B0
:1000B0005F0100085F0100085F0100085F010008A0
:1000C0005F0100085F0100085F0100085F01000890
:1000D0005F0100084D170008991700087D180008F7
:1000E0005F0100085F0100085F0100085F01000870
:1000F0005F0100085F0100085F0100085F01000860
:100100005F0100085F0100085F0100085F0100084F
:100110005F0100085F0100085F0100085F0100083F
:100120005F0100085F0100085F0100085F0100082F
:10013000DFF80CD000F018F800480047E51C000874
:10014000880800200648804706480047FEE7FEE78B
:10015000FEE7FEE7FEE7FEE7FEE7FEE7FEE7FEE777
:10016000ED16000831010008064C074D06E0E06876
:1001700040F0010394E8070098471034AC42F6D3EE
:10018000FFF7DAFFA01D0008C01D000800BFFEE752
:1001900010B502460B460020002104E0545C0444E4
:1001A000E0B24C1CE1B29942F8DBC443E0B2441C1B
:1001B000E0B210BD10B5354800780A281DD134488A
:1001C000007834490978884217D13148407831495C
:1001D0004978884211D12E48007A2E49097A8842FE
:1001E0000BD12B48407A2B49497A884205D12A48BD
:1001F000008840F40040284908802748008810F40F
:10020000004F42D0002025490870214800794870ED
:100210001F48407988701E488079C8701C48C07992
:100220000871084600781E4908701C4840784870DC
:100230001A48807888701948C078C87017480079C3
:100240000871012017490870174800686FEA00001C
:100250001649C1F880014FF40071154800F0F2FB17
:100260004FF4FA7001F0EAFC4FF40071104800F00E
:10027000E7FB0E48D0F88001C0430B4908604FF0FF
:100280000000024908700449088010BD07000020E2
:100290008C0100200E000020080000201800002023
:1002A0004000002045000020800122420000224240
:1002B0000010014010B588B046480078002831D0C1
:1002C000002044490870FC20434908701120487000
:1002D00042480078887041484078C8703F4880782C
:1002E00008713E48C07848713C4800798871072100
:1002F0003948FFF74DFF3849C87100203849086078
:100300004FF0FF024FF0E10100F0C4FD0823324A34
:10031000A821002000F080FD002000F045FC012015
:10032000304908702F480078002851D02E480068C6
:1003300000284DD1694600F001FD0446204601F039
:1003400021F904F04000402842D100208DF8070038
:10035000264800686FEA00002549C1F880014FF087
:100360000701684601F018F99DF801001B4909785A
:1003700088421FD19DF8020018494978884219D156
:100380009DF8030015498978884213D19DF804002F
:100390001249C97888420DD19DF805000F490979A5
:1003A000884207D100200F4908700E21114801F042
:1003B000F3F80DE000200A4908604FF00803064AF0
:1003C0004FF0A80100F028FD01200B49C1F8980169
:1003D00008B010BD450000201E0000204000002095
:1003E000988121423E0000200001214280012242EA
:1003F00000002242C00300200080214210B5D048F6
:1004000000780E281BD1CF48407BFB2817D1CD4860
:100410000078FA280DD1CA480078401EC949085C06
:10042000FB2806D1C848008840F40040C64908802F
:100430002DE00020C2490870C349088027E0C14868
:10044000007B1030BE490978884217D1BD4800783A
:10045000FA280DD1BA480078401EBA49085CFB283A
:1004600006D1B948008840F40040B74908800EE042
:100470000020B3490870B449088008E0B04800780B
:10048000182804DD0020AE490870AF490880AE4846
:10049000008810F4004F71D0AA488079AB49887168
:1004A000A848C179A948C171A648017AA748017234
:1004B000A448417AA5484172A248807AA34988722B
:1004C00008468079A2498871A048C179A048C171C5
:1004D0009E48017A9E4801729C48417A9C4841722C
:1004E0009A48807A78285FD012DC71283FD008DCE7
:1004F000212820D0222825D025282AD026287DD1A1
:100500002EE073283BD0742840D07528F7D144E002
:10051000A22874D008DC82284DD0942852D0A0287C
:1005200057D0A128EBD197E0A32869D0A42868D0A0
:10053000A528E4D1F2E087A001F058FB0020834910
:100540008872F3E085A001F051FB00207F4988729A
:10055000ECE086A001F04AFB00207C498872E5E0CF
:1005600086A001F043FB002078498872DEE087A076
:1005700001F03CFB002075498872D7E0DEE086A0E0
:1005800001F034FB002071498872CFE085A001F0B2
:100590002DFB00206D498872C8E085A001F026FB84
:1005A00000206A498872C1E084A001F01FFB00208E
:1005B00066498872BAE084A001F018FB0020634904
:1005C0008872B3E082A001F011FB00205F498872BD
:1005D000ACE05E488079824988715C48C179804886
:1005E000C1715A48017A7E4801725848417A7C4864
:1005F00041725648807A7A49887203E095E02FE08C
:100600007EE084E04F48407B504948734D48817BF1
:100610004E4881734B48C17B4C48C1734948017CAB
:100620004A4801744748417C48484174407B6D49C1
:1006300008704648807B48704448C07B88704348B7
:10064000007CC8704148407C0871012066490870F0
:1006500000203E49887269E000203C49887265E0CC
:100660003A488079614988713848C1795F48C171D9
:100670003648017A5D4801723448417A5B484172DC
:100680003248807A594988720120C872062008735E
:100690000020487356480178544881735448417883
:1006A0005248C17352488178504801745048C1780B
:1006B0004E4841744E4801794C48817402204B49A0
:1006C000C8740620087500204875464801784748D8
:1006D0008175444841784548C1754248817843480E
:1006E00001764048C178414841763E4801793F480B
:1006F00081761E2100F050FF00201449887215E019
:100700003CA001F073FA0020104988720EE03EA070
:1007100001F06CFA00200D49887207E03DA001F05D
:1007200065FA00200949887200E000BF00BF002080
:1007300005490880024908703B49087010BD000057
:1007400003000020C400002004000020F802002064
:100750009402002052657365740A00004765744670
:1007600069726D76657273696F6E0A0053657452B3
:10077000656164657249440A00000000476574526F
:10078000656164657249440A0000000044656C5765
:10079000686974650A0000004F70656E5768697477
:1007A000650A0000436C6F736557686974650A00D9
:1007B00041646457686974650A00000047657457AE
:1007C000686974650A00000048656172740A000077
:1007D000476574576869746553746174650A0000ED
:1007E000C003002040000020450000205C030020E2
:1007F000180000205570646174654669726D7665F5
:100800007273696F6E0A00005570646174654669A1
:10081000726D0A005570646174654669726D537437
:100820006174650A0000000002000020FA203B49C4
:100830000870102048700020887000213748C1706F
:100840000171417100203549887100213348C1711F
:100850000172417200203149C87400212F4801758E
:10086000FB202E494875FA202D4908701020487049
:100870000020887000212A48C17001714171002058
:100880002749887100212648C171017241720020F8
:10089000234981F84B000021214880F84C10FB20AF
:1008A0001F4981F84D00FA201E4908701020487039
:1008B0000020887000211B48C17001714171002027
:1008C0001849887100211748C171017241720020D6
:1008D0001449C876002113480177FB201149487755
:1008E000FA201149087010204870002088700021FB
:1008F0000D48C1700171417100200B4988710021C0
:100900000948C1710172417200200749C872002173
:1009100005480173FB200449487370479402002086
:10092000F80200205C030020C003002070472DE97E
:10093000F041024600250026002000230024002765
:1009400091F803C00CF00F0591F803C01CF0100FD4
:1009500003D091F802C04CEA050591F800C0BCF143
:10096000000F31D0146800202BE04FF0010C0CFA7E
:1009700000F3B1F800C00CEA03069E4220D18300C8
:100980004FF00F0C0CFA03F7BC4305FA03FC4CEADA
:10099000040491F803C0BCF1280F06D14FF0010CFC
:1009A0000CFA00FCC2F814C00AE091F803C0BCF1D4
:1009B000480F05D14FF0010C0CFA00FCC2F810C032
:1009C000401C0828D1D31460B1F800C0BCF1FF0F5F
:1009D00034DD546800202EE000F1080C4FF00108CF
:1009E00008FA0CF3B1F800C00CEA03069E4221D1CC
:1009F00083004FF00F0C0CFA03F7BC4305FA03FC1D
:100A00004CEA040491F803C0BCF1280F05D100F1B1
:100A1000080C08FA0CF8C2F8148091F803C0BCF175
:100A2000480F07D100F1080C4FF0010808FA0CF844
:100A3000C2F81080401C0828CED35460BDE8F08175
:100A4000416170470161704700BFFEE700BFFEE7EC
:100A5000704700007CB5054612A103C9CDE900012D
:100A60000821284600F064FD05236A463021284607
:100A700000F0D2F905236A461021284600F0F0F86C
:100A8000002406E01DF80400A52800D003E0601C47
:100A9000C4B2052CF6DB00BF052C01D001207CBDC3
:100AA0000020FCE7A5A5A5A5A500000008B501212B
:100AB0001C2000F0A7FA4020ADF8000010208DF8AF
:100AC000030003208DF8020069463148FFF72FFF2D
:100AD00040212F48FFF7B6FF1020ADF8000069460F
:100AE0002C48FFF724FF10212A48FFF7ABFF012015
:100AF000ADF8000048208DF8030003208DF80200B7
:100B000069462448FFF713FF4FF40070ADF800006A
:100B100010208DF8030003208DF8020069461C4860
:100B2000FFF705FF4FF400711948FFF78BFF4FF4F3
:100B30008050ADF8000069461548FFF7F8FE4FF405
:100B400080511348FFF77EFF4FF48070ADF800002E
:100B500048208DF8030003208DF8020069460C48F8
:100B6000FFF7E5FE00F012FC00F0CEFB00200A4982
:100B700008604FF001000949C1F890014FF00000F2
:100B8000074908604FF001000649C1F8B00108BDEF
:100B9000000C0140000801409881214200002142E0
:100BA000A48121420080214210B504461CB90020D6
:100BB0002749086002E00020264908604FF0010242
:100BC0004FF02301204600F065F90323224A2A2131
:100BD000204600F021F90323204A3021204600F06E
:100BE0001BF901222121204600F054F90122222183
:100BF000204600F04FF92A222521204600F04AF92C
:100C000007222621204600F045F90F222021204608
:100C100000F040F906223D21204600F03BF9012278
:100C20003C21204600F036F970222721204600F0B2
:100C300031F9FF22E221204600F02CF91CB90120F5
:100C40000349086002E001200249086010BD00006D
:100C500098812142A4812142991D0008941D000819
:100C60002DE9F0478046894615461E46B8F1000F2B
:100C700016D10020174908604946404600F004FCA0
:100C80000746002406E0FF21404600F0FDFB285502
:100C9000601CC4B2B442F6DB01200E49086015E0C6
:100CA00000200D4908604946404600F0EDFB07462C
:100CB000002406E0FF21404600F0E6FB2855601CBA
:100CC000C4B2B442F6DB0120034908603846BDE8EF
:100CD000F087000090012142B081214270B50546A5
:100CE0000E4685B90020114908603146284600F0BB
:100CF000CBFBFF21284600F0C7FB044601200C492E
:100D0000C1F890010FE000200A49086031462846EA
:100D100000F0BAFBFF21284600F0B6FB0446012094
:100D20000549C1F8B001204670BD00009001214284
:100D300000002142B08121420080214270B5064668
:100D40000D461021304600F0F3FB07213046FFF737
:100D5000C5FF044622462721304600F09BF814F0D8
:100D6000400F0AD007232A4661213046FFF778FF5B
:100D7000FF22E221304600F08DF8204670BD0000D1
:100D800010B504461CB900201F49086002E000208D
:100D90001E4908604FF001024FF02301204600F089
:100DA00079F803231A4A3021204600F035F803234E
:100DB000184A2A21204600F02FF80122212120463E
:100DC00000F068F801222221204600F063F81A2280
:100DD0002421204600F05EF82A222521204600F03A
:100DE00059F807222621204600F054F80E2220212F
:100DF000204600F04FF81CB901200349086002E0CA
:100E000001200249086010BD98812142A48121423D
:100E1000941D0008991D00082DE9F0478046894679
:100E200015461E46B8F1000F16D10020174908607C
:100E30004946404600F028FB0746002406E015F826
:100E4000011B404600F020FB601CC4B2B442F6DB3C
:100E500001200E49086015E000200D490860494650
:100E6000404600F011FB0746002406E015F8011B80
:100E7000404600F009FB601CC4B2B442F6DB01201E
:100E8000034908603846BDE8F08700009001214220
:100E9000B08121422DE9F04104460E46154684B941
:100EA0000020114908603146204600F0EDFA07465F
:100EB0002946204600F0E8FA01200C49C1F89001CB
:100EC0000FE000200A4908603146204600F0DCFAB5
:100ED00007462946204600F0D7FA01200549C1F807
:100EE000B0013846BDE8F081900121420000214266
:100EF000B08121420080214208B54FF4C06000F06B
:100F000065F826208DF8000001208DF801000220F0
:100F10008DF8020001208DF80300684600F01CF8EF
:100F200027208DF8000001208DF801008DF80200C7
:100F30008DF80300684600F00FF825208DF80000BA
:100F400000208DF8010001208DF802008DF80300CB
:100F5000684600F001F808BD70B5002100230F229B
:100F6000C4780CB3164C246804F4E064C4F5E0645F
:100F7000210AC1F10403CA40447804FA03F18478D9
:100F80001440214309010F4C0678A155047804F060
:100F90001F050124AC4005786D114FF0E02606EBEB
:100FA0008505C5F8004109E0047804F01F05012417
:100FB000AC40054D0678761145F8264070BD00001E
:100FC0000CED00E000E400E080E100E002490143B4
:100FD000024A1160704700000000FA050CED00E0C5
:100FE0007047000029B1064AD2690243044BDA6116
:100FF00004E0034AD2698243014BDA617047000082
:101000000010024029B1064A92690243044B9A61DA
:1010100004E0034A92698243014B9A6170470000E1
:101020000010024010B500F033F84FF4803000F0AB
:10103000F1F800F04DF90446012C1ED1002000F01B
:10104000DDF8002000F018F9A00200F009F94FF4D3
:10105000E011200400F022F9012000F019F900BF8E
:10106000392000F0A5F80028FAD0022000F024F979
:1010700000BF00F0BBF80828FBD1012144F20D00AD
:10108000FFF7C0FF01210220FFF7ACFF10BD0000F9
:101090000F48006840F001000D49086008464068AC
:1010A0000C4908400A494860084600680A49084057
:1010B000074908600846006820F480200860084658
:1010C000406820F4FE0048604FF41F0088607047BD
:1010D000001002400000FFF8FFFFF6FE30B50021CF
:1010E0000022002400232D4D6D6805F00C0121B174
:1010F000042905D0082923D105E0294D056022E007
:10110000274D05601FE0254D6D6805F47012234DD5
:101110006D6805F48034022505EB92421CB9214D1F
:10112000554305600BE01D4D6D6815F4003F03D07D
:101130001C4D5543056002E0194D5543056002E022
:10114000174D056000BF00BF144D6D6805F0F0013C
:101150000909154D6B5C0568DD4045600F4D6D68F4
:1011600005F4E061090A104D6B5C4568DD4085605F
:101170000A4D6D6805F46051C90A0B4D6B5C4568FA
:10118000DD40C560054D6D6805F44041890B074D94
:101190006B5CC568B5FBF3F5056130BD001002401E
:1011A00000127A0000093D00460000205600002091
:1011B00010B501460022002300204A11012A02D165
:1011C000094C236806E0022A02D1074C236A01E099
:1011D000054C636A01F01F02012494401C4201D0B7
:1011E000012000E0002010BD0010024002484068CD
:1011F00000F00C0070470000001002400146002083
:10120000034A506820F0F000084350607047000027
:10121000001002401149096821F480310F4A116021
:101220001146096821F480211160B0F5803F03D098
:10123000B0F5802F0ED106E00849096841F48031ED
:10124000064A116007E00549096841F4A021034AF4
:10125000116000E000BF00BF7047000000100240B6
:1012600001460020034A506820F4E06008435060C3
:10127000704700000010024001460020034A5068F9
:1012800020F4605040EAC1005060704700100240F6
:1012900001490866704700000000424202460020F3
:1012A000044B586820F47C1042EA01031843014BB8
:1012B000586070470010024001460020034A506801
:1012C00020F0030008435060704700000010024007
:1012D00038B5002000900024002500BF3120FFF722
:1012E00067FF05460098401C00900098B0F5A06F7D
:1012F00001D0002DF2D03120FFF75AFF08B10124B0
:1013000000E00024204638BD00B587B0012141F23D
:101310000500FFF777FEE020ADF8180018208DF8E3
:101320001B0003208DF81A0006A91648FFF7FFFAE4
:10133000E0211448FFF786FB0020ADF804004FF4CD
:101340008270ADF806000020ADF80800ADF80A0084
:10135000ADF80C004FF40070ADF80E001820ADF899
:1013600010000020ADF812000720ADF8140001A90C
:10137000054800F06BF80121034800F04DF807B074
:1013800000BD0000000801400030014000B587B0FA
:1013900001218803FFF726FE01210920FFF732FE15
:1013A0004FF46040ADF8180018208DF81B000320A2
:1013B0008DF81A0006A91648FFF7B9FA4FF46041F4
:1013C0001348FFF73FFB0020ADF804004FF4827094
:1013D000ADF806000020ADF80800ADF80A00ADF841
:1013E0000C004FF40070ADF80E001820ADF810009E
:1013F0000020ADF812000720ADF8140001A905483F
:1014000000F024F80121034800F006F807B000BD01
:10141000000C01400038004021B1028842F0400237
:10142000028004E002884FF6BF731A4002807047C2
:101430000246002013890B4201D0012000E0002069
:1014400070470146888970478181704710B5002236
:10145000028802F441520B884C8823438C88234332
:10146000CC8823430C8923434C8923438C89234311
:10147000CC8923431A430280838B4FF2FF742340AD
:1014800083830B8A038210BD2DE9F04106460F4687
:1014900026BB06E0601CC4B2C82C02DB0020BDE8FD
:1014A000F08102212048FFF7C3FF0028F2D039461F
:1014B0001D48FFF7C9FF002405E0601CC4B2C82C1A
:1014C00001DB0020EBE701211748FFF7B1FF0028FF
:1014D000F3D01548FFF7B5FFC5B222E005E0601C68
:1014E000C4B2C82C01DB0020D9E702210F48FFF766
:1014F0009FFF0028F3D039460C48FFF7A5FF0024D2
:1015000005E0601CC4B2C82C01DB0020C7E7012144
:101510000648FFF78DFF0028F3D00448FFF791FF3E
:10152000C5B22846BBE7000000300140003800404B
:1015300070B505460C467DB90F4800884FF6C77157
:1015400008400D4908800846008820430880012192
:101550000A48FFF761FF0EE0084800884FF6C771A0
:101560000840064908800846008820430880012179
:101570000248FFF751FF70BD0030014000380040C5
:101580007047000010B504460249204600F010F8EC
:1015900010BD00000038014070B504460D46034AF6
:1015A0002946204600F014F870BD000000380140C4
:1015B00070B504460D4600BF8021284600F042FA6F
:1015C0000028F9D02146284600F009FB012070BD13
:1015D0002DE9F04104460D46164614B90120BDE838
:1015E000F0810AE014F8017B31463846FFF7E0FF4E
:1015F00008B90020F3E7681E85B2002DF2D1012062
:10160000EDE710B500F002F810BD00000CB50020A9
:10161000019000903248006840F480303049086002
:1016200000BF2F48006800F4003000900198401C73
:101630000190009818B90198B0F5A06FF1D1284831
:10164000006810F4003F02D00120009001E000206B
:1016500000900098012842D12248006840F0100014
:10166000204908600846006820F00300086008462A
:10167000006840F002000860194840681849486056
:101680000846406848600846406840F4806048600A
:101690000846406820F47C1048600846406840F4E2
:1016A000E81048600846006840F08070086000BF9D
:1016B0000B48006810F0007FFAD00948406820F01D
:1016C0000300074948600846406840F0020048604F
:1016D00000BF0348406800F00C000828F9D10CBD99
:1016E00000100240002002407047000010B513486F
:1016F000006840F001001149086008464068104940
:1017000008400E494860084600680E4908400B49E9
:1017100008600846006820F4802008600846406899
:1017200020F4FE0048604FF41F008860FFF769FF57
:101730004FF000600449086010BD00000010024036
:101740000000FFF8FFFFF6FE08ED00E010B540F2E4
:1017500025510D4800F083F9A8B140F225510A48FF
:1017600000F0C7F8084800F035FAC4B2214607482F
:1017700000F035FA064807490978445405480078CE
:10178000401C0449087010BD00380140004400406E
:10179000C40000200300002010B540F2255112487B
:1017A00000F05DF988B140F225510F4800F0A1F832
:1017B0000D4800F00FFAC4B20C480D4909784454A2
:1017C0000B480078401C0A4908700821064800F0C0
:1017D00039F9012806D10821034800F081F80248B0
:1017E00000F0F8F910BD0000004400405402002051
:1017F0000B00002010B586B0044601210520FFF73C
:1018000001FC01214804FFF7EDFB0420ADF81400B2
:1018100003208DF8160018208DF8170005A915482B
:10182000FFF785F80820ADF8140004208DF81700A4
:1018300005A91048FFF77BF801940020ADF80800D7
:10184000ADF80A00ADF80C00ADF810000C20ADF8B2
:101850000E0001A9084800F051F9012240F225517B
:10186000054800F026F90121034800F051F806B0C0
:1018700010BD0000000801400044004010B540F2D7
:101880002551144800F0EBF8B0B140F22551114851
:1018900000F02FF80F4800F09DF9C4B20E480F4930
:1018A000097844540D480078401C0C4908700846DB
:1018B000007800F00F0008700821064800F0C2F818
:1018C000012806D10821034800F00AF8014800F079
:1018D00081F910BD004800408C0100200700002065
:1018E00001F40072B2F5007F00D100BFCA4302804C
:1018F000704710B500220023A1F510646A3C00D1A6
:1019000000BF0A1201249440A3B2DC43048010BD3E
:1019100021B1828942F40052828104E082894DF62D
:10192000FF731A408281704700B585B0012144F2EF
:101930000400FFF767FB4FF40070ADF800000320D0
:101940008DF8020018208DF8030069463948FEF72B
:10195000EEFF4FF48060ADF8000004208DF8030026
:1019600069463448FEF7E3FF4FF4E1300190002070
:10197000ADF80800ADF80A00ADF80C00ADF81000A5
:101980000C20ADF80E0001A92B4800F0B7F8012299
:1019900040F22551284800F08CF801212648FFF735
:1019A000B7FF01218804FFF71DFB01210820FFF785
:1019B00029FB4FF48060ADF8000003208DF8020091
:1019C00018208DF8030069461C48FEF7B0FF4FF45D
:1019D0000060ADF8000004208DF803006946174848
:1019E000FEF7A5FF4FF4965001900020ADF80800D7
:1019F000ADF80A00ADF80C00ADF810000C20ADF801
:101A00000E0001A90E4800F079F801A90C4800F079
:101A100075F8012240F22551094800F04AF80121E9
:101A20000748FFF775FF40210348FFF759FF05B04E
:101A300000BD00000008014000380140000C0140DA
:101A40000048004002460020B1F5007F00D100BFF1
:101A500013880B4201D0012000E00020704770B5D0
:101A600002460024002300250020A1F510666A3EEE
:101A700000D100BFC1F3421501F01F03012606FA91
:101A800003F3012D02D19689334006E0022D02D1E5
:101A9000168A334001E0968A33400C12012606FA7A
:101AA00004F41688344013B10CB1012000E000208A
:101AB00070BDF0B503460024002600250020A1F5E6
:101AC00010676A3F00D100BF1846C1F3421401F00D
:101AD0001F06012707FA06F5012C01D10C3004E09E
:101AE000022C01D1103000E014301AB107682F43E6
:101AF000076002E00768AF430760F0BD2DE9F047DB
:101B000086B005460E460024A24600BFA146002727
:101B1000B08900B100BF2F462C8A4CF6FF700440FC
:101B2000F08804432C82AC894EF6F3100440B08850
:101B300031890843718908430443AC81AC8A4FF66C
:101B4000FF400440B0890443AC8201A8FFF7C6FA05
:101B50001F48874202D1DDF810A001E0DDF80CA09B
:101B6000A88910F4004F08D00AEBCA0000EB0A1055
:101B700031684900B0FBF1F807E00AEBCA0000EB5E
:101B80000A1031688900B0FBF1F86420B8FBF0F06E
:101B900004012009642101FB1089A88910F4004F79
:101BA00008D0322000EBC900B0FBF1F000F00700D4
:101BB000044308E0322000EB09106421B0FBF1F08F
:101BC00000F00F0004432C8106B0BDE8F087000050
:101BD0000038014001468888C0F308007047C1F30F
:101BE00008028280704700BFFEE70000014A0249F8
:101BF00000F013B8691C00085C00002002E008C86F
:101C0000121F08C1002AFAD170477047002001E076
:101C100001C1121F002AFBD170472DE9F041164681
:101C20000F460446002503E03946B0476D1C641C8E
:101C300020780028F8D12846BDE8F08110B502468A
:101C40000BE0C82007E0122101E04B1E99B20029E9
:101C5000FBDC431E98B20028F5DC1300A2F101045E
:101C6000A2B2EED110BD000070B504460D46E0B240
:101C70000549088000BF40210348001FFFF7E2FE2E
:101C80000028F8D0204670BD0438014008B5012175
:101C90001020FFF7B7F90120ADF8000010208DF8F3
:101CA000030003208DF8020069460D48FEF73FFE51
:101CB00001210B48FEF7C6FE4FF40070ADF800009E
:101CC00010208DF8030003208DF8020069460448B7
:101CD000FEF72DFE4FF400710148FEF7B1FE08BD7E
:101CE00000100140FFF79EF9FFF706F9FFF7CEFF5E
:101CF000FFF71AFE4FF4E130FFF77CFDFEF7D6FE4A
:101D000002E019A0FFF772FF0020FEF7A3FE0028F3
:101D1000F7D102E014A0FFF769FF0120FEF79AFE59
:101D20000028F7D1FEF782FD134800686FEA000033
:101D30001249C1F880014FF4FA70FFF77FFF0F4896
:101D4000D0F88001C0430D49C1F880010CA0FFF715
:101D50004DFF0120FFF714F805E0FEF72BFAFEF720
:101D6000A9FAFEF74BFBF8E754686520322E34479A
:101D7000204572726F7221008001224200002242CF
:101D8000303033D0B4C2EBC8EDBCFEB2E2CAD40DE1
:101D90000A00000034431010013443101001000009
:101DA000C01D00080000002060000000FC1B0008AF
:101DB000201E000860000020280800000C1C0008FD
:101DC0000000000000000000000000000000D1D171
:101DD000E0D000000000D2D200000000000031324C
:101DE000333435363738393132333435363738399C
:101DF00000000000000000000000000000000000E3
:101E000000000000000000000000010203040102C5
:101E10000304060708090204060800000000000089
:0400000508000131BD
:00000001FF
